:0E29FF00C104C100C103C101C1024108075E4D
:103651009005D3E0FCA3E0FD9005D2E025E024E451
:10366100F582E43405F58322900724E0FBA3E0FA18
:10367100A3E0F9020D90900807E0FF900784E06F46
:1036810022900785E0FFA3E0FDA3E0FB229005D394
:103691007422F0A3742EF02224A5F582E43406F5F9
:0236A100832282
:103E7700AE8475840F75A40F7580F075A7F0E4FD07
:103E8700FC0DBD00010CBC4EF8BD20F5E58030E609
:103E970004E4FF800CE5B0540F70047F018002E456
:033EA700FF8E8407
:013EAA0022F5
:10118E0090071E12111500000000E4900722F09047
:10119E000727F0A3F075FFDE75FFADF5E6F5E71254
:1011AE003C5ED2AFC203E49005CFF0124312E4903E
:1011BE000729F0900729E0FFD39403500DE4FD12A8
:1011CE004489900729E004F080E975840F123E3DB2
:1011DE001215EED204D20075840F12214A9006A980
:1011EE00E0B401111235A4900723EFF0E012369906
:1011FE007401F0800690072374FFF01218C7900652
:10120E00A9E064017026900723121658120D90B4AF
:10121E00020A900723E0FF1238D18010123669B40B
:10122E00010A900723E0FF7D01123CD8E4900729C4
:10123E00F0900729E0FFD39403504F900723E0FE70
:10124E00EF6E6046900729121658900729E0FF129C
:10125E003699E06401701D123669B402051238D158
:10126E00801F123669B40119900729E0FFE4FD12C0
:10127E003CD8800D1236697008900729E0FF1234B1
:10128E003A900729E004F002123F1243B9EF7003BF
:10129E000214CA123B17EFB4180040030214C19097
:1012AE0012B4F82828730212FC02132E0213400205
:1012BE00134402134802135002135402135802131C
:1012CE005C0213640213C20213CA0213D30213F098
:1012DE000214120214560214A10214A50214A90239
:1012EE0014AD0214B10214B80213210214BF30015E
:1012FE0015A203B39203300309C20ED20212442187
:10130E00800CC20280083002051244E7C202D204E9
:10131E000214C1900807E0FF7D011242800214C141
:10132E009005D1E004F0E075F00384E5F0F0E4FF01
:10133E00800A7F0180067F0280027F03123116022F
:10134E0014C1E4FF800A7F0180067F0280027F03C2
:06135E001243740214C1E9
:101364009005D2E090072AF004F090072AE0C39495
:10137400155023E0FF12365DE0FCA3E0FDEF25E00D
:1013840024E2F582E43405F583ECF0A3EDF0900754
:101394002AE004F080D4E490060CF0A3F01236594D
:1013A400E0FFA3E09005D3CFF0A3EFF0123659E0AD
:0E13B400FCA3E0FDE4FF123A8D123DC9804912
:1013C2001223851244218041900612E0F4F00214A7
:1013D2004C9005D2E0D3940050030214C19005D280
:1013E200E014F012365C12163A124421801B90056A
:1013F200D2E0C3941440030214C19005D2E004F079
:1014020012365C12163A124421D200D2040214C1DE
:10141200D39005D4E094269005D3E0942A40077433
:101422002AF0A37426F0D39005D4E0942E9005D32D
:10143200E0942250030214C1A3E024F6F09005D3F5
:10144200E034FFF0123651121669124421D204D24E
:10145200000214C19005D3E07002A3E070031236BB
:101462008E9005D3E0FEA3E0FFC3942EEE942250AB
:101472000512368E8017D3EF941CEE942A504090BA
:1014820005D4E0240AF09005D3E03400F01236517E
:10149200121669124421D204D20012442180207F04
:1014A20001800E7F0180117F0280067F0280097F0A
:1014B20003122D0680097F03122C6E800280FE1219
:1014C20043B9EF60030212A1123F44EF7003021509
:1014D200D8900783E06431701E123677701912417A
:1014E200D150FB121626A3E0900705F01227E61250
:1014F20041D150FB12164F900783E06432701812EC
:10150200367770131241D150FB12162612271A1287
:1015120041D150FB12164F900783E0642D702F12B9
:101522003677702A1241D150FB900807E0FF124330
:10153200E41241D150FB1236821229531241D1508A
:10154200FB900807E0FF1243CFE4900784F0900776
:1015520083E0642E702A12367770251241D150FB37
:10156200900807E0FF1243E41241D150FB12368289
:1015720012289F1241D150FB900807E0FF1243CF7F
:10158200900783E0FFB41406D203D202D204EFB470
:101592001506C203C202D204EFB40B06D201D20373
:1015A200D202300331EF14601B04702A900784E0EA
:1015B200FFC3941E50209005CFEFF01215EED2001B
:1015C200D2048012900784E0FFC3941E5008900555
:1015D200CFEFF01244E7300405121BF2C2042000E0
:0C15E200030211E5122A9CC2000211E570
:1015EE001243F99005D3E0FCA3E0FDE4FF123A8D1F
:1015FE009005D8E0FCA3E0FD7F01123A8D9005DD49
:10160E00E0FCA3E0FD7F02123A8D9005E2E0FCA320
:10161E00E0FD7F03123A8D22900807E0FF1243E4AB
:10162E00900785E0FFA3E0FDA3E0FB22E0FEA3E030
:10163E00FF9005D3EEF0FCA3EFF0FDE4FF123A8D20
:10164E0022900807E0FF1243CF22E0FF123EDF9008
:10165E000724EBF0A3EAF0A3E9F022ECF0A3EDF0FF
:09166E00E4FF123A8D1237E72265
:102A0D004506A500000000004A06AA0000000000CF
:102A1D0000000000004506B4FFFFFFFFFF4A06B9A6
:102A2D000000000000000000000041069FE8450680
:062A3D00A00000000000F3
:10396A0090081FE024A5F582E434062290081FE09F
:10397A0024B4F582E43406F583E0229007B5E02505
:10398A00E024B9F582E43406F5832225E024AAF579
:10399A0082E43406F58322F074A02CF582E434061E
:0B39AA00229007B61211099007B62208
:10214A0090069FE0603BE490081FF090081FE0FFB4
:10215A0025E02456F582E43407F583E0FCA3E0FD8C
:10216A00EF25E0245AF582E43407F583ECF0A3ED79
:10217A00F090081FE004F0E0B402D090069FE0144B
:10218A00F090069FE070047D0180027D00E4FF125A
:10219A001EC890069FE070047D0180027D007F01C9
:1021AA00121EC8E490081FF090081FE0FFD39404A1
:1021BA004003022268EF123995E0FEA3E0FFD394B0
:1021CA0096EE9400401F123976D3940F406B900814
:1021DA001FE0FD12396EF5837403F074B42DF58295
:1021EA00E43406805012396AF583E0FDB4032C907A
:1021FA00081FE0FC24A0F582E43406F583E004120B
:10220A0039A1F583E0D3940F402F90081FE0FC1208
:10221A00396EF58374011239A1801AEDB4010A12DC
:10222A00396AF5837402F08010C3EF9430EE94009B
:10223A00500712396AF583E4F090081FE0FF12395B
:10224A0095E4F0A3F074B42F12397CC394145005AA
:0E225A0012397604F090081FE004F00221B261
:012268002253
:1040B600AE84E4F5848FBBFF0FEFB40AFBC2EDD2EA
:1040C600EC30EDFD900809E5BFF0A3E5BEF0AF06C4
:0A40D6008F84900809E0FEA3E0FFCC
:0140E00022BD
:103B9F00AE84ADE775840253E7FBE5E85401FC8F73
:103BAF00BBE4FF0FEFB40AFBC2EDD2EC30EDFDE446
:103BBF0090080BF0A3E5BEF053E8FEAF04EC42E82B
:103BCF00AF058FE7AF068F8490080BE0FEA3E0FFF1
:013BDF0022C3
:05434400E0FCA3E0FD18
:10434900D3EF9DEC6480F8EE648098400122AE04BE
:03435900AF05228B
:031A060002201D9E
:10201D00C0E0C0F0C083C082C0D075D000C000C089
:0D202D0001C002C003C004C005C006C0070A
:0F203A009007B5E4F09007B5E0FFD39404506130
:102049001240B6E4FCFDC004C005C006C007123941
:1020590085E0FEA3E0FFE47B0FFAF9F8120F8ED0BA
:1020690003D002D001D000EF2BFFEE3AFEED39FD8F
:10207900EC38FC1239ABE0FCA3E0FDA3E0FEA3E0E1
:10208900FF78041210C11239ABA3A3E0FEA3E0FF4D
:08209900123985EEF0A3EFF00F
:1020A1009007B5E004F002203F7F07123B9F9006A6
:1020B100AA1243449006AAEEF0A3EFF07F06123B6A
:1020C1009F9006AC1243449006ACEEF0A3EFF07F74
:1020D10005123B9F9006AE1243449006AEEEF0A36C
:1020E100EFF07F04123B9F9006B01243449006B07C
:1020F100EEF0A3EFF07F051240B6EF7804CEA2E731
:1021010013CE13D8F8FF9006B21243449006B2EEF4
:10211100F0A3EFF07F061240B6900756EEF0A3EF62
:0E212100F07F071240B6900758EEF0A3EFF0E3
:10212F00D007D006D005D004D003D002D001D00004
:0B213F00D0D0D082D083D0F0D0E032AE
:031A36000244FF68
:0444FF0053E7F3325A
:062A4300C10941067515F2
:1040E100E0FEA3E0FFED25E0244BF582E43406F584
:1040F100832290079AE0FBA3E0FAA3E0F922EF25DF
:0B410100E024E4F582E43405F583229D
:10257F00900797EEF0A3EFF0A3EDF0A3EBF0A3EA33
:04258F00F0A3E9F0DC
:102593007EFFE4FCFD1240F38D82758300120DA9CA
:1025A300FFC39E5004AE07AC050DEDB415E7AF06AF
:1025B300900799E0C39F500302264DEC1240E7E0D9
:1025C300FEA3E0D39400EE9400404BAD04EDC3941E
:1025D300145030ED25E0244DF582E43406F58312E2
:1025E30040E1EEF0A3EFF0ED2401FFE433FE1240EF
:1025F300F38F828E83120DA98D82758300120E3D97
:102603000D80CA1240E6E4F0A3F01240F38D827508
:102613008300E4120E3DAF04AD07EDC39415502AB9
:102623001240E6E0FEA3E04E701D9007971240E1D2
:10263300EEF0A3EFF0900799E0FFA31240F68D822E
:0A264300758300EF020E3D0D80D0FC
:01264D00226A
:10238500D209122A9CE49006D8F09006D8E0FFC343
:102395009415501C74C32FF582E43406F583E4F0DC
:1023A500EF1240E7E4F0A3F09006D8E004F080DAFD
:1023B5007D2E7C22E4FF123A8D1243A29006DDEEBB
:1023C50080389006DAE0704FA3E0FEA3E0FFC390EB
:1023D50006DEE09F9006DDE09E503C1244E0AD072E
:1023E5009006DBE0FEA3E0FF7B017A0679C31225A8
:1023F5007F9006DBE0FFA3E0A3CFF0A3EFF07D0124
:10240500E4FF1232B69006DAEFF01243A29006DB33
:10241500EEF0A3EFF080AB9006D87401F09006D8EB
:10242500E0FF25E02449F582E43406F583E0FCA3CA
:10243500E0FD1240FFECF0A3EDF09006D8E004F0CB
:10244500E0B416D99005E47422F0A3742EF0C20905
:0F245500E49006D9F09006D9E0FFD394035035F8
:10246400123EDF9006DFEBF0A3EAF0A3E9F0900060
:1024740002120DA9FF60169006DF1240F61240FF0B
:0D248400E0FFA3E0900003CF8FF0120F6186
:0E2491009006D9E004F080C1123DC9022A9CD9
:103DC9007D14EDFF3395E0FEEF25E0FFEE33FE7441
:103DD900E42FF58274053EF583E0FEA3E0FF4E6013
:013DE9000FCA
:0F3DEA0090080DEEF0A3EFF0900675EDF0FF22BC
:093DF900DDD0E4900675F0E0FF56
:013E0200229D
:022A4900C18A40
:10423E00120E7190080FEEF0A3EFF0C322EAFF7E8C
:10424E00007C00020E5F74022AF582E43404F583CA
:01425E00223D
:0E1A0900E4FFFE0FBF00010EEF64644E70F5A7
:011A170022AC
:1044470020F907E59A30E7F880F98F9B30FFFDC226
:02445700FF2242
:023AD300AC073E
:103AD500A984ABE6AAE7E4F584F5E6F5E70CC29020
:103AE500121A09EDC4540FFFAE04EEC454F04FFF93
:103AF500124447AF05EFC454F0FF124447121A09A8
:103B0500D290121A09AF018F84AF038FE6AF028FEF
:013B1500E7C8
:013B1600228C
:02302D00AA07F0
:10302F00300A0C7FFF900402E4F0A3DFFCC20A1207
:10303F004254E0FF600122EAC3941950107DB4128C
:10304F00424B7D1912423E74FF9FFB8049EAC394A5
:10305F003350107D1812424B7D1A12423E74629FFC
:10306F00FB8033EAC3947FEA5015FF7E007C007D1E
:10307F001D120E5F7D4C12423E74479FFB801775E9
:10308F00F003A4FFE5F0C4F854F0C8EFC4540F48A0
:0C309F00FFC374309FFB124254EBF0FFA3
:0130AB002202
:0E448900A907AF0512302DAD07AF01023AD3DF
:102A4B004406EA000000004406EE030303034406B9
:052A5B00E20000000094
:103F1200900820E0FF24EAF582E43406F583E022EB
:103F2200900820E024EEF582E43406F58322FFEEC9
:103F3200F0A3EFF0900820E024E2F582E43406F5E5
:023F42008322D8
:1018C700E4900820F0123F12FC74A52FF582E4344F
:1018D70006F583E0B40119123F22E4F074EA2FF50C
:1018E70082E43406F583E4F074E22F123F3CE4F01F
:1018F700900820E0FF123F26E0FD704D74EA2F129A
:101907003F19C394FF502B900756E0FEA3E07806DB
:10191700CEC313CE13D8F99006E6123F30E0FB048E
:10192700F0EB6F7001EE60030219D3123F1204024D
:1019370019C2900612E09008206009123F25740230
:10194700F00219D3E024EE8020EDB40225900820A0
:10195700E0FF24A5F582E43406F583E06402606CB9
:101967009006A9E0706674EE2F123F287401F0020A
:1019770019D3900820E0FF123F26E06401704D90D4
:101987000758E07003A3E0F4604274EA2F123F198E
:10199700D394004031900758E0FEA3E07806CEC309
:1019A70013CE13D8F99006E8123F30E0FD04F0EDAE
:1019B700B50719E4B50615123F1214F074E22F1299
:1019C7003F3CE4F08006123F227403F0900820E0C9
:1019D700123F17FD6C600A900820E0FF124489D27D
:1019E70004900820E004F0E0D3940350030218CCDD
:0119F70022CD
:1041F7009007CAE0FBA3E0FAA3E0F92225E024E454
:10420700F582E43405F583E022E50A850B83850C06
:04421700826401229A
:1042DC007F80900502E4F0A3DFFC7B017A05790274
:0C42EC008B0A8A0B890C8A088909D2B55C
:0142F80022A3
:1043B900124210700AE50965827004E50865837088
:0643C90002FF227F012229
:103B1700124210700AE50965827004E50865837032
:103B270003FF802FAB0A050CE50CAA0B7002050BEF
:103B370014F9120D90FF74019005826B700AE50C61
:103B470065827004E50B65837009750A01750B05BD
:033B5700750C02E8
:013B5A002248
:031A03000235FCAD
:1035FC00C0E0C083C082C0D075D000C004C006C07B
:01360C0007B6
:10360D00AF8475840FE5B0541FFE0509E509AC08BC
:10361D007002050814F5828C83EEF0C3E5099482DF
:10362D00E50894054006750805750902C2B5308692
:05363D00FDD2B58F84F1
:0F364200D007D006D004D0D0D082D083D0E032D1
:053116009007C9EFF075
:10311B00123EDF9007CAEBF0A3EAF0A3E9F09007A9
:10312B00C9E0FF6011A31241FA900001120DA9F43E
:10313B00900001120E3D1241F7900001120DA97083
:10314B002B900002120DA9FE6022124203FCA3E099
:10315B00FD123A8D1241F7900002120DA912420393
:10316B00FFA3E0900003CF8FF0120F61124421D226
:03317B0004D2007B
:01317E00222E
:10437400123EDF7401120DD6B40304E4120E2B12A4
:064384004421D204D20026
:01438A002210
:103BE000E475F001120EC685F082F58322EEF0A393
:103BF000EFF0A3ECF0A3EDF0A3EAF0A3EBF022AF1B
:103C000001AE027C00E4FDA302110908F6E4F5848C
:103C1000C2AF43B70122E0FEA3E0AA06F97B01226E
:103D15009007BAE584F0A2AF920B123BFF9007BD66
:103D2500E0FEA3E0780DA606123C0B438F02438FFD
:103D35000118E6FE08E6F5828E83E4F053B7FEF53A
:0B3D45008FA20B92AF9007BAE0F5844C
:013D50002250
:05391E0090079DEDF093
:10392300A3E584F0A2AF920C123BFF90079DE0FF4A
:10393300FD3395E0FCEDF44C60229007A1E0FCA37D
:10394300E0780FA604123C0B758F0118E6FC08E61D
:10395300F5828C83EFF053B7FEE4F58FA20C92AFA0
:0639630090079EE0F584D0
:01396900223B
:103747009007A3123BED9007A7E07002A3E060404B
:103757009007A3123C16A3E0FEA3E0F5828E83E058
:10376700FD12391E9007A8E024FFF09007A7E03468
:10377700FFF09007A6E004F070069007A5E004F0BC
:103787009007A4E004F070BE9007A3E004F080B6B1
:01379700220F
:0844C900E4900000F0A3F022D2
:10421B00900000123C16123D15900000E0FEA3E04A
:10422B00FF7C007D021B7A04123747E4900000F0FC
:03423B00A3F022CB
:0D2EA700900768EDF0900766EEF0A3EFF0E5
:102EB400EE54FCFE900000E0FCA3E0FD7002EE6C1A
:102EC4006047ED4C600312421B900766E0FEEE542F
:102ED400FCFE7F00900000F0A3EFF0900769EEF095
:102EE400A3EFF0A37400F0A37402F07FFF7E0390BD
:102EF4000769123BE0E493FD90076B123BE0EDF0B1
:102F0400EF1F70011EEF4E70E6900768E0FF900718
:102F140066E0FCA3E0FDEC5403FC74022DF582741E
:062F2400003CF583EFF014
:012F2A002284
:103FD4009007A9123BED9007AD74FFF5F0120EC6E1
:103FE40045F0601A9007A9E475F001120EC6AFF00F
:0F3FF400FE9007AB123BE0E0FD122EA780D82213
:10325000E4FFFE75840F438C670FBF00010EBE0BA9
:10326000F8BFB8F5E58C30E7FB43890453A1DFE4F0
:10327000F58475B73075840F43A120438901758D9E
:1032800001758F01758E04FEFF0FBF00010EEF6404
:103290000F4E70F5438902E58920E4130FBF00014A
:1032A0000EBE0FF3BFFFF0E4F58443EF1080E87526
:0532B0009702E4F58A1D
:0132B50022F6
:1041AB00AF8475840F75E10343E20443E3C075A448
:1041BB000F7580F075A50775AD0775A6FF75A0FF88
:0541CB0075A7E08F84E0
:0141D00022CC
:0D449700AF84E4F58475D48475D1038F845F
:0144A40022F5
:10440E00AF84E4F584759D0443F809759A40D2F89B
:02441E008F8489
:014420002279
:0F446B00E4F584758810758902F584758E022238
:101A1B00AF84758401E4F5C975CA3C75CB5D75CD92
:081A2B006E75CCACF5C88F8488
:011A33002290
:1042F900AF84758402E4F5C975CA1975CBFF75CD0C
:08430900FF75CC19F5C88F8483
:014311002289
:10425F00AF84E4F584F5BA75BC9875E8807584026F
:10426F00F5BA75BCF975E88075C4AF75C6FF8F8454
:01427F00221C
:10438B00AF8443E70143E70443F704D2A8D2A9E47F
:06439B00F584D2888F8436
:0143A10022F9
:103C5E009008117427F0A37410F090081174FFF5FA
:0F3C6E00F0120EC6FED3E5F09400EE940050EB7A
:103C7D001232501241AB123C9B12440E1244971259
:0E3C8D0042DC12425F12446B12317F02438B05
:104003009007C0E0FBA3E0FAA3E0F9A3E075F00298
:10401300A4F58285F08322E014F0E0C364809480E9
:0E40230022EFF0A3EBF0A3EAF0A3E9F0A32252
:021A340000228E
:1042A000C2A57F027E001242BEC2A67F037E00121C
:0E42B00042BED2A57F037E001242BED2A622DD
:0531E800900813EFF058
:1031ED00123248C2A6123248C2A59008147407F0D4
:1031FD00C2A57F037E001242BE900814E0FF900826
:10320D0013E0FEA807088002C313D8FC1392A67F13
:10321D000312323990081412401A50D4C2A5D2A606
:0B322D007F0212323930A603121A345F
:10323800227E001242BED2A57F037E001242BE2229
:083248007F037E001242BE224A
:0536A300900815EFF096
:1036A800A37407F0C2A57F037E001242BE900816DD
:1036B800E0FF900815E0FEA807088002C313D8FCB5
:1036C8001392A61236E490081612401A50D6C2A5D4
:0B36D800D2A61236E430A603121A340A
:1036E300227F027E001242BED2A57F037E001242D9
:0236F300BE22F5
:053497009007F5EFF0C5
:10349C00E49007F7F09007F67407F0C2A5D2A67F68
:1034AC00037E001242BE1234E19007F7E025E0FFE4
:1034BC00A2A6E4334FF09007F612401A50DDC2A5D5
:1034CC009007F5E07004D2A68002C2A61234E190F7
:0434DC0007F7E0FF0F
:1034E000227F027E001242BED2A57F037E001242DE
:0234F000BE22FA
:033E03009007BF66
:103E06001240247402F07F201231E8124003120E91
:103E1600DCE5F0FF1236A3124003120EDCFF123669
:103E2600A39007C3E004540FFFF09007BFE00454CB
:073E36000FB507D70242A0FF
:0330AC0090074E3C
:0B30AF00124024740AF07F211231E867
:1030BA007F01123497900753E4F0A3EFF090075280
:1030CA00E0FF90074EE0C39FFF123497900755EF39
:1030DA00F0FD900754E0FE7C00E42DFFEC3EFE90EC
:1030EA00074FE0FBA3E0FAA3E0F9A3E0FD124010CA
:0F30FA00EE8FF0120F61ED04540FFF900752F0AC
:0D31090090074EE004540FB507A70242A046
:103EAB00900747E0FBA3E0FAA3E0F9900746E07523
:103EBB00F002A4F58285F08322FFE0F9A3E0FAA3D8
:103ECB00E0900747C9F0A3EAF0A3E9F022D2A57F5F
:043EDB00197E00222A
:0D44B300A2B7300D01B350030080F50022C8
:1039B50053A6BFD2A69007F8740FF0C2A57F197E53
:1039C500001242BE123ED81242BE9007FAE025E030
:1039D500FF9007F9E033FEA2A6E433FDEF4DFFEEBD
:1039E500F0A3EFF09007F8E014F0E0C36480948052
:0A39F50050C99007F9E0FEA3E0FFBF
:0139FF0022A5
:083A47009007FBEEF0A3EFF085
:103A4F00ED14A3F09007FDE0FFC364809480402D38
:103A5F00C2A59007FBE0FEA3E0A807088005CEC330
:103A6F0013CE13D8F91392A67F197E001242BE12FD
:0D3A7F003ED81242BE9007FDE014F080C753
:013A8C002217
:0B264E00900744EFF0A3EDF0A3EBF0C9
:1026590090074CE584F0A3E5E1F075840F43A640AB
:10266900900745E0B40106A3E024E0800690074600
:10267900E024C0FEE43390074AF0A3CEF09007446B
:10268900E0FF7002C2A0EFB40102C2A1EFB40202DE
:10269900C2A2EFB40302C2A390074AE0FEA3E0FF7F
:1026A9007D09123A47900745E0B4010C1239B51279
:1026B9003EABEE8FF0120F61900745E0700E123EAF
:1026C900AB120EDCFFAEF07D10123A47C2A57F05B2
:1026D9007E001242BE900744E0FF7002D2A0EFB420
:1026E9000102D2A1EFB40202D2A2EFB40302D2A333
:1026F9007F147E001242BE123ED81242BEC2A553BA
:10270900A6BFD2A690074DE0F5E190074CE0F5840D
:01271900229D
:0A3D510090076DEFF090076FEBF0A4
:103D5B00900773EDF0EB04540F90076FF090076D25
:103D6B00E0900770123EC4900773E0FB7D011226B2
:103D7B004E900773E004540FFFF090076FE0B50708
:013D8B00DC5B
:013D8C002214
:0A3D8D00900774EFF0900776EBF05A
:103D970090077AEDF0EB04540F900776F0900774D4
:103DA700E0900777123EC490077AE0FBE4FD122605
:103DB7004E90077AE004540FFFF0900776E0B507BE
:013DC700DC1F
:013DC80022D8
:0E2A60004407560000000044075A0000000022
:102D9900E0F8A3E0F9A3E0FAA3E0FB123B5B90069D
:102DA900F61211099006F2E025E02456F582E43482
:102DB90007F583E022F583E0FEA3E0FBC374FF9BE4
:102DC900FF740F9EFEE49400FDE49400FC22E47F6E
:102DD90001FEFDFCE0F8A3E0F9A3E0FAA3E0FB2281
:102DE9009006F2E025E0240EF582E434062225E07F
:102DF900245AF582E4340722E47BFF7A0FF9F8229A
:102E0900E0FCA3E0FDA3E0FEA3E0FF22F583EEF0E2
:082E1900A3EFF09006F3E022A4
:081EC8009006F2EFF0A3EDF02B
:101ED000E4A3F0A3F09006F2E0FD122DF7F583E005
:101EE000FEA3E0FFED122DB1FCA3E0C39FFDEC9E2D
:101EF000FCC3ED9440EC6480948040089006F4E4C8
:101F0000F0A304F0D3ED94C0EC6480947F50087487
:101F1000FF9006F4F0A3F09006F4E0FCA3E0FD4C83
:0D1F2000700302201CEDF47002ECF47064FC
:101F2D00FCFD9006FE1211099006FE122DD7C3126C
:101F3D0010AB500A9006FE12111500000001122D73
:101F4D00E9F583E0FEA3E0FFE4FCFD122E02120F83
:101F5D008E9006FE122D99FEA3E0FFE4FCFD900687
:101F6D00F6122DDD120F8E9006FA121109122E01A6
:101F7D009006FA122E09123B5B122DE9122E1560F6
:011F8D0077DC
:0F1F8E000220029006F4E07004A3E06401706882
:101F9D00122DE9122DBE122E01120F8E9006F61281
:101FAD0011099006F2E0122DF7122DBE9006FA12CD
:101FBD0011099006FA122DD7C31210AB500A9006D4
:101FCD00FA121115000000019006F6122E09A31247
:101FDD002D99122DC19006F6122DDD120F8E122E97
:101FED0001123B5BC374FF9FFF740F9EFE122DE920
:081FFD00122E156003124421AD
:102005009006F2E0FF122DB1FCA3E0FDEF122DF7D3
:07201500F583ECF0A3EDF0F0
:01201C0022A1
:0D2A6E004A072B7E306D79335B5F707F7BF4
:1034F200900819E0FEA3E0FF7C007D0A120E7174B1
:103502002B2DF58274073CF58322E0FEA3E0FF7CBD
:10351200007D0A120E71900819EE227E00900819A1
:10352200EEF0A3EFF022242BF582E43407F583E0DA
:10353200FB22A3E0FF900819E422FFE05480FDEF94
:093542004D22E0FB7A007D01221C
:101BF200900817E5E6F0A3E5E7F0E4F5841219F89A
:101C0200E4F5E6F5E7C291FD7C03900735E4F0A325
:101C1200DCFC7C007D03200303300207900737E0E1
:101C22004401F0900612E06007900737E04402F0AA
:101C32009005D0E0FFB40109900737E04404F0803A
:101C42000BEFB40207900737E04408F09005D1E0AB
:101C5200FF7009900737E04410F0800BEFB40107E2
:101C6200900737E04420F0E4FF74EA2FF582E43471
:101C720006F583E06015900736E0FE7401A80708B8
:101C82008002C333D8FC4E900736F00FEFB404D96C
:101C92009005D6E09007367006E04420F08004E01C
:101CA2004410F09005D5E0FFB40109900736E044F6
:101CB20080F0800BEFB40207900736E04440F090CA
:101CC20005E0E09007357006E04402F08004E0444D
:101CD20001F09005DFE0FFB40109900735E0440808
:101CE200F0800BEFB40207900735E04404F0900552
:101CF200DBE09007357006E04420F08004E04410F9
:101D0200F09005DAE0FFB40109900735E04480F075
:101D1200800BEFB40207900735E04440F0E4FCFD8D
:101D220053F87FE59A20E7FB74352DF58274073C62
:101D3200F583E0F59BE4FFFE0FBF00010EEF641494
:101D42004E70F50DBD00010CED64034C70D2D291C2
:0A1D5200900817E0F5E6A3E0F5E7BE
:011D5C002264
:0A19F8007F03900735E4F0A3DFFC45
:011A020022C1
:05331A009007FEEFF03A
:10331F00E4F9A3F0A3F09007FFE0FEA3E0FFC3944E
:10332F0008EE64809480504374017E00A8070880E3
:10333F0005C333CE33CED8F9FF9007FEE0FDE4FE90
:10334F00EF5DFFA3A3E0FDC374079DFDEFA8050884
:10335F008005C333CE33CED8F949F9900800E00485
:0D336F00F070B39007FFE004F080ABAF01F9
:01337C00222E
:102F2B0090077BEEF0A3EFF0A3EDF0A3EAF0A3EB99
:012F3B00F0A5
:102F3C00A3E5E6F0A3E5E7F0AF84E4F584C292FEE6
:102F4C00EEFD90077BE07003A3E06D702553F87FD6
:102F5C00E59A20E7FB90077DE0F59BE4F909E9B4DD
:102F6C0014FB90077EA3E0F59BE4F909E9B414FB8C
:102F7C00801A53F87FE59A20E7FBE4F59BF909E901
:102F8C00B414FBE4F59BF909E9B414FB0EEEB4039D
:0F2F9C00AFD292900780E0F5E6A3E0F5E78F84CF
:012FAB002203
:102E21007B1F7A007D05122E827B3E7D06122E9736
:102E31007B4E7D01122E827B377D02122E977B0EF7
:102E41007D03122E9F7B777D04122E9F7D01122E12
:102E51008A900732E0FB7D027F017E00122F2B7DDD
:102E610003122E8A7B4F7D047F017E00122F2B7C63
:102E710001AD04E4FBFAFFFE122F2B0CECB409F1B7
:102E8100227F027E00122F2B2290072DE0FB7F0173
:102E91007E00122F2B227F027E00122F2B227F0217
:062EA1007E00122F2B221F
:10317F00E4900821F0900821E0FFC3940350307EC3
:10318F0000E4FBFA7D0F122F2B0B7D0C1231D9FFB0
:10319F007E001B7D09122F2B900821E0FF7E007D02
:1031AF000A122F2B7B077D0B1231D904F080C6E456
:1031BF00900821F0900821E0FFD39403500B1237B1
:0931CF0098900821E004F080EB67
:1031D80022900821E0FF7E00122F2B900821E02288
:102A9C0030096B7B5B7A007D01122B257B4E7D020E
:102AAC00122B257B777D037F027E00122F2B1B7D43
:102ABC00047F027E00122F2BE4FB7D057F02FE12A9
:102ACC002F2BE47D067F02FE122F2B90082274011F
:102ADC00F0900822E0FDD39404500AE4FBFA7F0145
:102AEC00122B2D80EC9008227401F0900822E0FD4E
:102AFC00D394085023E4FBFAFF122B2D80EDE490C5
:102B0C000822F0900822E0FFD39403500B121677A2
:082B1C00900822E004F080EBB8
:102B2400227F027E00122F2B22FE122F2B900822CE
:042B3400E004F022A7
:10167700EF14607B14700302174414700302178879
:10168700240360030217D09005D2E075F00A84FFA7
:1016970012351D1235287A007D057F02122F2B90F7
:1016A70005D2E075F00A84AFF012351D1235287D9A
:1016B700067F02122F2B9005D312350CF0A3EFF003
:1016C7001234FAE07D04121805E044807D031218F5
:1016D700057F0212183612351F4E7008FB7D017FF9
:1016E700020217841234F21235447F0202173F9028
:1016F70005D6E0700512353480069005D812350CF2
:10170700F0A3EFF01234F2E0FB7A007D0412184FD9
:10171700E09005D612353CFB7D0312184F7F01126E
:10172700183612351F4E7008FB7D017F01021784A2
:101737001234F21235447F017E000217CD9005DB8B
:10174700E0700512353480069005DD12350CF0A3E4
:10175700EFF01234F27D041217D19005DB12353CFD
:101767007D031218977D0212187F12351F4E7005E0
:10177700FB7D0180071234F2123544E4FFFE0217A5
:10178700CD9005E0E0700512353480069005E21231
:10179700350CF0A3EFF01234F27D081217D1FF9049
:1017A70005E012353D7D071218977D0612187F1246
:1017B700351F4E7005FB7D05800A1234F2E0FB7A77
:0917C700007D05E4FFFE122F2B4A
:1017D00022E0FB7A00E4FFFE122F2B900819E0FEB6
:1017E000A3E0FF7C007D0A120E71900819EEF0A3B1
:1017F000EFF07C007D0A120E71742B2DF5827407B8
:101800003CF583E022FB7F027E00122F2B9008190B
:10181000E0FEA3E0FF7C007D0A120E71900819EE35
:10182000F0A3EFF07C007D0A120E71742B2DF5826F
:1018300074073CF58322E0FB7D027E00122F2B9083
:101840000819E0FEA3E0FF7C007D0A120E71227FE2
:10185000017E00122F2B900819E0FEA3E0FF7C0010
:101860007D0A120E71900819EEF0A3EFF07C007D56
:101870000A120E71742B2DF58274073CF58322E059
:10188000FBE4FFFE122F2B900819E0FEA3E0FF7C83
:10189000007D0A120E7122FBE4FFFE122F2B90082E
:1018A00019E0FEA3E0FF7C007D0A120E719008197A
:1018B000EEF0A3EFF07C007D0A120E71742B2DF573
:0718C0008274073CF583224E
:10379800EF14601514601D146023240370277C0146
:1037A8007F021237DBB409F8227C017F011237DB74
:1037B800B405F8227C011237CEB405FA227C051232
:0537C80037CEB409FA40
:1037CD0022AD04E4FBFAFFFE122F2B0CEC22AD040C
:0A37DD00E4FBFAFE122F2B0CEC2285
:05410C00900761EDF0D9
:10411100AF01AB0790076274FF1210D6EC4D4E4F02
:104121006010900761E08B828A83F00BBB00010A6B
:0241310080E22A
:014133002269
:10435C0074EA2BF582E43406F583E02274EE2BF537
:08436C0082E43406F583E0222F
:1035A40079FF7FFF7EFFE4FD7CFFFB12435C700329
:1035B400AF03220BEBB404F3E4FB124368B4010C35
:1035C40012435CF9C39E5004AF03AE010BEBB40489
:1035D400E9EFF4600122E4FB124368700C12435CCF
:1035E400FFD39C4004AD03AC070BEBB404EAEDF449
:0735F4006003AF05227F0018
:0135FB0022AD
:1042800090081BEFF0A3EDF07F0A1233DD90081BBE
:10429000E0FF1233DD90081CE0FF1233DD0244A57D
:0844D1007F021233DD0244A555
:063F44001244EDEF6027BE
:103F4A0090081D7407F0A37482F012403190081D86
:103F5A00E475F001120EC685F082F583EFF0124483
:073F6A00F3EF70E67F012276
:033F71007F0022AC
:1043CF00900823EFF07F2F1233DD900823E0FF12C8
:0543DF0033DD0244A5DE
:1043E400900824EFF07F301233DD900824E0FF12B0
:0543F40033DD0244A5C9
:072A7B004206130043C10EE7
:101D5D0090800075F043ED121146EC75F043A4250B
:101D6D0083AF8290070EF0A3EFF0900706E0900787
:101D7D000B75F043A42400F9748035F0FA74FFF06C
:101D8D00A3EAF0A3E9F02290070BA3E475F001128A
:101D9D000EC690070EFEAFF0E475F001120EC6856B
:101DAD00F082F583E49322E075F043A42400F582DC
:101DBD00E5F03480AF8222E5C0F0A3E5CFF0A3E5D6
:101DCD00C3F0A3E584F0E4F58475C04475CF8F436B
:101DDD00C3019005CF740FF0229005CFE075F0434D
:101DED00A42400F9748035F0FA22900825E025E04E
:101DFD0024E4F582E43405F58322E024FFFFE43486
:101E0D00FFFE900707E0FCA3E0FD22900583A3E40D
:101E1D0075F001020EC6E024FFFEE434FF900707C3
:101E2D00F0A3CEF0229005CDE0FCA3E0FDC39443DA
:101E3D00EC9400229005D3E0FEA3E0FF22C39007AF
:101E4D000AE09443900709E0940022E0F5C0A3E076
:101E5D00F5CFA3E0F5C3C2C622AD04EDFFEEF0A3AE
:101E6D00EFF022EBF0AC07A2AFE433A3F0AF052205
:101E7D00900003742275F02E020F61EEF0FCA3EFBB
:101E8D00F0FD22E49005CDF0A3F02274882DF582AB
:101E9D00E43405F58322FE7C057DD07B437A002258
:101EAD009FEE6480F8EC648098229005CDE004F0FC
:0B1EBD0022E4F0A3EFF0E07F00FE2223
:102FAC00E4900825F0900825E0FFD394155038EFF5
:102FBC00121DFBE0FEA3E0FFC3942EEE9422500CF6
:102FCC00121DF77422F0A3742EF08013D3EF942605
:102FDC00EE942A400A121DF7742AF0A37426F0907E
:102FEC000825E004F080BEE4900825F0900825E068
:102FFC00FFD39403502A123EDF900003120EDCFF25
:10300C00AEF0C3942EEE942250028009D3EF942696
:10301C00EE942A4003121E7D900825E004F080CC2B
:01302C002281
:1037E7009005D2E0FF9005D7E0B5070E121E419075
:1037F70005D8121E887F01123A8D9005D2E0FF90FE
:1038070005DCE0B5070E121E419005DD121E887F0C
:1038170002123A8D9005D2E0FF9005E1E0B5070E60
:0F382700121E419005E2121E887F03123A8D2275
:102B38009007CD7401F0E4A3F0A3F0A3F01244C908
:102B48007E877FDA7C077DCD7B017A00123FD4E453
:102B58009007CFF09007CFE0FFD394035023123EA5
:102B6800DF7401120E2BF582758300E4120E3D907E
:102B78000002E4120E3D121E7D9007CFE004F080A3
:102B8800D3E490060EF0A3F0900612F0900610F031
:102B9800A3F0D200D2049007CEF09007CEE0FFC396
:102BA800941E501575F043EF121DB8121EA3123F64
:102BB800D49007CEE004F080E17E877FDB7C077D40
:0B2BC800D07B017A00123FD402421BB8
:10442100200E0F3001083003071244D18002D2025E
:03443100D20E2286
:104312009087DBE493600C9087DAE4936401600396
:09432200122B38E49005CFF022C3
:1043F900121DE67BFF78D07C057D017E007F43128C
:054409000D6AC20E2245
:104459001244C99005CF121DB4121EA3123FD402F3
:02446900421BF4
:0644E700124459C20E222E
:034503000244E788
:0A27E600900703EDF0900702EFF0FA
:1027F000D39B404F121E23EB14900706F090070363
:10280000121E07D3121EAD4003022893121D5DE471
:10281000900709F0A3F0121D9412289470069007F7
:1028200009E004F0121E4A40ED12421B900708E036
:1028300004F07006900707E004F0900706E004F04B
:102840000227FD900703121E23900705E014A3F052
:10285000900702121E07C3121EAD4037121D5DE421
:10286000900709F0A3F0121D9412289470069007A7
:1028700009E004F0121E4A40ED12421B900708E0E6
:1028800024FFF0900707E034FFF0900706E014F013
:03289000022850CB
:0C28930022FD122EA790070AE004F0229C
:05271A00900582EDF0C6
:10271F00EF149005CBF0EB14A3F0900582E014FFBB
:10272F009005CBE0D39F40030227DAA3121DB4FE1E
:10273F00121E90121E3250210FEFAA0670010E14B6
:10274F00F5828A83E493FB121E98EBF09005CEE09E
:10275F0004F070DF121EB780DA9005CCE09005838D
:10276F00121D7E9005CB121DB4900586F0A3EFF0DD
:10277F00121E90121E18900586121DA21227DB70D2
:10278F0003121EB7C39005CEE094439005CDE0949D
:10279F000040E09005CB121DE9900583121D8A12AF
:1027AF001E90121E325014121E18FEAFF0121E98F9
:1027BF00E01227DB70EC121EB780E712421B900568
:0B27CF00CBE004F0A3E004F002272997
:0C27DA0022FD122EA79005CEE004F02294
:03289F009007108F
:1028A200121E70A3121EBE900712F0A3EFF0900743
:1028B20012121E66C2AF90071A121DC41244C91228
:1028C2001DE6900716121D8AE4900714F0A3F090FB
:1028D2000712E0FCA3E0FFECFD900710E0FBE490A0
:1028E20007D4F0D20512249F900719EFF0FD90074C
:1028F20016121E1BFEAFF0122EA7900713E004F073
:102902007006900712E004F0900715E004F07006DC
:10291200900714E004F0C3900715E0944390071465
:10292200E0940040AA12421B9005CFE004F0E0C3FD
:10293200941E408890071DE0F58490071A121E58D5
:10294200123C9BD2C6123C9B900711E024FF92AF2F
:012952002262
:03295300900738B2
:10295600121E7090073C121EBE90073CF0A3EFF0CB
:1029660090073C121E66C2AF900740121DC4900528
:10297600CFE0FFC3941E506775F043EF121DB89069
:10298600073EF0A3EFF0E490073AF0A3F090073C7F
:10299600E0FCA3E0FFECFD900738E0FB90073E1259
:1029A6001DA59007D4F0C20512249F90073DE004B0
:1029B600F0700690073CE004F090073BE004F070EE
:1029C6000690073AE004F0C390073BE09443900773
:1029D6003AE0940040B79005CFE004F002297490E5
:1029E6000743E0F584900740121E58123C9BD2C65E
:0829F600900739E024FF92AFC5
:0129FE0022B6
:07249F009007D1EFF0A90541
:1024A600C20620C3FD20C5FAC2C4D2C5E4FFFD3072
:1024B600C3FD30C3FDE5C154F8FC64086004ECB408
:1024C6001013EFB40105EB44018003EB54FEF5C293
:1024D6007D0102256DECB4180B89C27D02C2C4C20F
:1024E600C502256DECB420028045EC6428703CEDF5
:1024F600B4020E9007D1E0F5C27D03C2C5C2C48006
:1025060066EDB4031B300508D2C57F01C2C48057EF
:102516009007D4E0F5C2C2C57D04E4FFC2C480477B
:10252600ED64047042D2C47D05803CECB4300AD21E
:10253600C4D2C57D08E4FF802EECB438028024ECBA
:10254600B44006C2C2C2C5801EECB448028014EC78
:10255600B450028004ECB4580AD2C47D07AEC2C29D
:10256600C28004D2C4D2C5C2C3ED64076008ED645C
:082576000560030224B8AF0662
:01257E00223A
:0A2A820041061D0041063600C108A0
:1036F500900620E475F001120EC685F082F583224E
:103705009006207406F0A37437F02290061BE0FFA4
:10371500A3E09006172290061BE0FEA3E0FF9006AB
:1037250017227E067F4B900617E022E0F5C2900631
:1037350017E06E22900618E004F022900617E004C8
:02374500F02270
:1041D10012371BE0FCA3E0FDB50719ECB5061590FD
:1041E1000620E0FEA3E0FFEDB50709ECB5060520CA
:0641F100C502D322C32227
:10432B00AF84E4F58475C04475CFE2C2C343E602A3
:08433B0043F60275C3038F84F1
:014343002257
:103C9B007E067F22900619EEF0A3EFF090061EEE43
:103CAB00F0A3EFF0900615EEF0A3EFF07E067F3752
:103CBB0090061BEEF0A3EFF0900620EEF0A3EFF0D2
:0D3CCB00900617EEF0A3EFF0C20702432BA6
:1041840090061E1236F8EFF090061E1236F8EDF087
:1041940090061EE0B4060FA3E0B4360A90061E741F
:0741A40006F0A37422F022D3
:0D44A500AF84E4F584C207C2C4D2C58F8481
:0144B20022E7
:1033DD0020072FD2071236F574FFF07C067D4B9037
:1033ED000620E0B50408A3E0B50503123705123633
:1033FD00F5E4F0900620E0B50408A3E0B50503124E
:10340D0037051236F5E4F0900620E0B40608A3E087
:10341D00B44B031237051236F5EFF0900620E0B4E9
:0D342D000608A3E0B44B031237057F01220F
:10405E00900619E0FCA3E0FD900615E0B50408A358
:10406E00E0B505037F0022900619E0FCA3E0F5827F
:0C407E008C83E0B507037F01227F002245
:1040310090061AE004F07006900619E004F090066C
:10404100191236F8E0FF900619E0B4060FA3E0B4A8
:0C405100360A9006197406F0A37422F0E1
:01405D002240
:0644ED007FFF12405E2279
:0644F300E4FF12405E220E
:031A1800021A3976
:101A3900C0E0C0F0C083C082C0D075D000C000C073
:101A490004C005C006C007E5C154F81211521BB6FF
:101A5900001A94081A94101AC5181AF4201AFA28A8
:101A69001B5F301B64381B6E501B70581B7C601B3E
:101A790072681B7C701B72781B82801B8B881B828F
:101A8900901B8B981B9EA000001BDBC2C512373927
:101A99007003123740123727B5060BA3E0B50706C6
:101AA9009006171237089006171236F81237307059
:101AB90003A3E06F6003021BDB021B561237397068
:101AC90003123740123727B5060BA3E0B507069076
:101AD90006171237089006171236F81237307003B6
:101AE900A3E06F6003021BDB021B56123710CF8085
:101AF9001690062012371EE0FCA3E0FDB50713EC93
:101B0900B5060F90061BEEF0A3EFF0C2C5D2C402D2
:101B19001BDB8D828C83E0B4FF07C2C4D2C5021BD4
:101B2900DB1237397003123740123727B5060BA37A
:101B3900E0B507069006171237089006171236F80F
:101B49001237307003A3E06F6003021BDB900617A6
:101B5900123708021BDB1237108031123710CFF011
:101B6900A3EFF0806D80128010123710CFF0A3EF31
:101B7900F0D208ADC27FFF8004ADC2E4FF124184F8
:101B89008050900615E0FFA3E090061ECFF0A3EF6A
:101B9900F0D2C4803D90061EE0FFA3E0900615CF69
:101BA900F0A3EFF030082BD2C5C208802512371BED
:101BB900EEF0A3EFF0900615E0FDA3E090061ECD30
:101BC900F0A3EDF0D2C4A3E06E7003A3E06F60024E
:101BD900D2C5C2C3D007D006D005D004D000D0D01A
:091BE900D082D083D0F0D0E032AC
:03000000020C00EF
:03000300021A03DB
:03000B00021A06D0
:03001300021A09C5
:03001B00021A0CBA
:03002300021A0FAF
:03002B00021A12A4
:03003300021A1599
:03003B00021A188E
:03004300021A1B83
:03004B00021A1E78
:03005300021A216D
:03005B00021A2462
:03006300021A2757
:03006B00021A2A4C
:03007300021A2D41
:03007B00021A3036
:03008300021A332B
:03008B00021A3620
:03009300021A3915
:03009B00021A3C0A
:0300A300021A3FFF
:100C0000787FE4F6D8FD9000007F007E20E4F0A31A
:0A0C1000DFFCDEFA758121020C55AD
:0644F900140A05140A0577
:0F2A8C0041069E00480676000000000000000092
:102269009007DEE0FBA3E0FAA3E0F9900002120D6B
:10227900A925E024E4F582E43405F583E0229007FA
:10228900EAE0FBA3E0FAA3E0F990000222EFF012E2
:102299003EDFA3EBF0A3EAF0A3E9F0229007EDE01B
:1022A900FF900003120EDCFDACF0229007E512113D
:1022B900099007E5E0FCA3E0FDA3E0FEA3E0227D91
:1022C900017BFF7E007F03120D6A900688A3E0FD63
:1022D9005430FFE4C4F854F0C8EFC4540F4822FF47
:1022E900A3E0900003CF8FF0020F61900804E0256E
:1022F900E02476F582E43406F58322E0FBA3E0FAD4
:10230900A3E0F9900003120EDCFFAEF0C3942EEEA9
:1023190094222290078EE0FEA3E0FFC322EF25E07E
:1023290024B9F582E43406F583E0FEA3E022FEE455
:102339003DFDE43CFC021109F0900828E0FF7B0216
:102349007D02227422F0A3742EF022FFE47B7A7AB4
:102359000FF9F802101904F0A37406F0A3747EF0C3
:1023690022EEF0A3EFF0E4A3F0A3F0229007B1125C
:0C23790011099007B122900001020DA98B
:10413400900826EBF090069EE0700E90077712230D
:104144005F900826E0FB023D8D900826E0FF7B018E
:084154007A06797E123E032277
:05354B00900827EFF0DD
:103550007F2090067EE4F0A3DFFC900682E4F0A3D7
:1035600004F0900827122345124134E4900686F0B7
:10357000A3F0A3E4F0E04412F0A3E0F0E054CFF0B5
:103580004410F0900827E0FF7B057D041241347F52
:10359000027E00123FA4900827E0FF7B0FE4FD129B
:0335A000415C008B
:0135A3002205
:0744D9007F557E00023FA4A5
:10388400900802EDF0A3EBF0900801EFF07B0FE459
:10389400FD12415C900803E09006826009E0444018
:1038A400F0A3E0F08004E054BFF0900689E054F007
:1038B400F0900802E0540FFF900688E0F0A3E04F78
:0D38C400F0900801E0FF7B057D0202413419
:10443400EF9006826008E04420F0A3E0F022E0540C
:03444400DFF02284
:0D2BD3009007C5ECF0A3EDF09007C4EFF003
:102BE0007B0FE4FD12415C9007C5E07002A3E0702A
:102BF000069007C512234C9007C512231F94B0EE10
:102C0000941D400912337D9007C7EE80099007C5D7
:102C1000E0FFA3E0A3CFF0A3EFF09007C7E044806C
:102C2000FFA3E0900684CFF0A3EF122C60122C4F8C
:102C300030E6FA900684E0547F122C60122C4FA3E9
:0F2C400020E6F99007C4E0FF7B0B7D0B02415C9F
:102C4F009007C4E0FF7B0A7D0A12415C900692E078
:0F2C5F0022F09007C4E0FF7B037D031241342273
:0B3A8D00900804EFF0A3ECF0A3EDF0B4
:103A9800EF1222F8E0FEA3E06D7002EE6C602B904E
:103AA8000804E0FFA3E0FCA3E0FD122BD31222F4EC
:103AB800E0FEA3E04E7003123DC9900805E0FEA3A6
:0A3AC800E0FF1222F4EEF0A3EFF08D
:013AD20022D1
:1032B600900828EFF0ED9006826009E04402F0A342
:1032C600E0F08004E054FDF0900682E04401F0A3B3
:1032D600E012234112413412330D900692E030E69B
:1032E600F6900682E054FE12234112413412330D49
:1032F600900692E0A320E6F5900828E0FF7B0B7D80
:103306000B12415C7F0022900828E0FF7B0A7D0AB1
:0433160012415C22E2
:1043A2007B0B7D0BE4FF12415C900694E05403FE0C
:0743B200A3E0FF12383622E0
:0744E000900692A3E0FF2209
:0944C000900692A3E0FF7E0022A9
:033F74009007D5DE
:103F770012236A9007D512231F9007D8E09F900756
:103F8700D7E09E50177FF47E011242BE9007D8E01B
:0C3F970004F070DF9007D7E004F080D742
:013FA30022FB
:08337D00900789EEF0A3EFF0C8
:10338500788B7C077A4479F91222C8FBED54C090FA
:10339500078E700512234C8007741DF0A374B0F0DE
:1033A50012231C90078AE09F900789E09E500890A1
:1033B5000789EEF0A3EFF012231C90078AE09FFF28
:1033C500900789E09EFE748B2BF582E43407F58324
:0733D500E0FD7C00120E7107
:0133DC0022CE
:0442BE00AD07AC0696
:1042C2007B01EDAE047805CEC313CE13D8F9FFEB14
:0942D200D39FE49E50030B80E928
:0142DB0022C0
:033FA4009007D9AA
:103FA70012236A9007D912231F9007DCE09F90071E
:103FB700DBE09E50177FE87E03123F749007DCE03A
:0C3FC70004F070DF9007DBE004F080D70E
:013FD30022CB
:10415C00900829EBF090069EE0700E9007701223E9
:10416C005F900829E0FB023D51900829E0FF7B019C
:08417C007A06797E1230AC22B4
:103C200090082AE584F075840F43A640D2A5C2A06F
:103C3000C2A1C2A2C2A3C2A6C2A47F647E00123FD8
:103C400074D2A47F647E00123F74D2A0D2A1D2A20B
:0D3C5000D2A353A6BFD2A690082AE0F584A7
:013C5D002244
:08383600900790EEF0A3EFF003
:10383E0078927C077A4479FC1222C8FFED54C0902E
:10384E000795700512234C8007741DF0A374B0F019
:10385E0074922FF582E43407F583E0FF7E00900723
:10386E0090E0FCA3E0FD120E5F900796E02FFF9014
:05387E000795E03EFE8D
:013883002222
:103E3D00123C20E490082BF090082BE0FFD3940364
:103E4D00502712379890082BE0FF12354B90082B16
:103E5D00E0FF7B017D0F12388490082BE0FF1216D6
:093E6D007790082BE004F080CFEF
:013E76002229
:103EDF007B007A007900EF14601214601714601CD5
:103EEF002403701E7B017A0579D080167B017A0539
:103EFF0079D5800E7B017A0579DA80067B017A0508
:023F0F0079DF58
:013F1100228D
:0338D1009007DD80
:1038D4001222969000027401120DF8900002120D4B
:1038E400A9FF900675E0FD3395E0FCC3EF9DEC6401
:1038F40080F8748098400B9007DE12228A740112BB
:103904000E3D122269FCA3E0FD9007DDE0FF123AB0
:093914008D1222691222E8D20092
:01391D002287
:033CD8009007E171
:103CDB00122296ED60047F0480059007E1E0FF124D
:103CEB00408A9007E212228AEF120E3D9007E212F1
:103CFB00226CFCA3E0FD9007E1E0FF123A8D9007E8
:093D0B00E212226C1222E8D2003F
:013D1400228C
:10408A00122326FFE4FCFD7B14FAF9F8120F8E12B4
:10409A0022B41223541222B42401FFE43E9007E50D
:0B40AA001223379007E5A3A3A3E0FF5B
:0140B50022E8
:103A00009007AF7407F0A374F8F0122326FBAA0600
:103A1000E4F9F89007AFE0FEA3E0FFE4FCFD120F2D
:103A20008E1223751222BD1223541223751222BD49
:103A3000242EFFEE34229007B11223379007B1A352
:063A4000A3E0FEA3E0FF7D
:013A4600225D
:0F447A007C007D0A120E717C007D0A120E5F22FB
:03343A009007E90F
:10343D0012229612237F701B9007E9E0FF12408A3B
:10344D00122287EF120E3D122274FFA3E0900003AB
:10345D00CF8021122287E4120E3D9007E9E0FF1282
:10346D003A0012447A9007EAE0FBA3E0FAA3E0F9F0
:10347D00900003EE8FF0120F619007E91222A8124F
:09348D003A8D124421D204D20050
:013496002213
:032D06009007ED46
:102D090012229612237F70369007EE12228A120D34
:102D1900A9FFD3941440079000027414800AEFD3DA
:102D290094009000025004E4020E3D74FF120DF865
:102D39001222741222E81222A5123A8D804A9007B3
:102D4900EE122304500A900003742275F02E8011AC
:102D5900D3EF9426EE942A400B900003742A75F061
:102D690026020F61C3EF9438EE94224022900003AB
:102D790074FF75F0F6120F141222A5123A8D9007FE
:0F2D8900EE12228AE4120E3D124421D204D2002F
:012D98002218
:032C6E009007F1DB
:102C710012229612237F70399007F212228A120DC6
:102C8100A9FFC3941440079000027414800AEFC393
:102C910094009000025004E4020E3D7401120DF8FC
:102CA1001222741222E89007F11222A8123A8D80A2
:102CB1004C9007F2122304500A900003742275F01D
:102CC1002E8011C3EF9426EE942A400B90000374DA
:102CD1002A75F026020F61D3EF941CEE942A50243A
:102CE100900003E475F00A120F149007F11222A864
:102CF100123A8D9007F212228AE4120E3D124421FB
:042D0100D204D20026
:012D050022AB
:100C1A0002118EE493A3F8E493A34003F68001F251
:100C2A0008DFF48029E493A3F85407240CC8C333DB
:100C3A00C4540F4420C8834004F456800146F6DFAA
:100C4A00E4800B01020408102040809029FFE47E12
:100C5A00019360BCA3FF543F30E509541FFEE4939F
:100C6A00A360010ECF54C025E060A840B8E493A366
:100C7A00FAE493A3F8E493A3C8C582C8CAC583CA91
:100C8A00F0A3C8C582C8CAC583CADFE9DEE780BE49
:012A9B00003A
:100C9A00E709F608DFFA8046E709F208DFFA803E3C
:100CAA0088828C83E709F0A3DFFA8032E309F60829
:100CBA00DFFA8078E309F208DFFA807088828C8391
:100CCA00E309F0A3DFFA806489828A83E0A3F60845
:100CDA00DFFA805889828A83E0A3F208DFFA804C1F
:100CEA0080D280FA80C680D4806980F280338010F6
:100CFA0080A680EA809A80A880DA80E280CA80335F
:100D0A0089828A83ECFAE493A3C8C582C8CCC583D6
:100D1A00CCF0A3C8C582C8CCC583CCDFE9DEE780A6
:100D2A000D89828A83E493A3F608DFF9ECFAA9F025
:100D3A00EDFB2289828A83ECFAE0A3C8C582C8CC7B
:100D4A00C583CCF0A3C8C582C8CCC583CCDFEADE94
:100D5A00E880DB89828A83E493A3F208DFF980CCF6
:100D6A0088F0EF60010E4E60C388F0ED2402B404EF
:100D7A000050B9F582EB2402B4040050AF23234596
:060D8A008223900CEA73C5
:100D9000BB010689828A83E0225002E722BBFE0261
:090DA000E32289828A83E4932294
:100DA900BB010CE58229F582E5833AF583E02250FF
:100DB90006E92582F8E622BBFE06E92582F8E22249
:0D0DC900E58229F582E5833AF583E4932263
:100DD600BB010989828A83F8E028F022500327F7AD
:100DE60022BBFE05F8E328F3228A838982F8E4937E
:020DF6002822B1
:100DF800BB010FF8E58229F582E5833AF583E028FF
:100E0800F0225009C58229F8E58226F622BBFE09A0
:100E1800C58229F8E22582F222F8EA2583F583E9DA
:030E2800932822EA
:100E2B00BB010689828A83F0225002F722BBFE01A6
:020E3B00F322A0
:100E3D00F8BB010DE58229F582E5833AF583E8F0EB
:100E4D00225006E92582C8F622BBFE05E92582C897
:020E5D00F2227F
:100E5F00EF8DF0A4A8F0CF8CF0A428CE8DF0A42EA7
:020E6F00FE2261
:100E7100BC000BBE0029EF8DF084FFADF022E4CC65
:100E8100F875F008EF2FFFEE33FEEC33FCEE9DEC2E
:100E9100984005FCEE9DFE0FD5F0E9E4CEFD22ED74
:100EA100F8F5F0EE8420D21CFEADF075F008EF2FBE
:100EB100FFED33FD4007985006D5F0F222C398FDAF
:050EC1000FD5F0EA224C
:100EC600A3F8E0C5F025F0F0E582158270021583DF
:060ED600E0C838F0E8223C
:100EDC00BB0110E58229F582E5833AF583E0F5F054
:100EEC00A3E0225009E92582F886F008E622BBFE31
:100EFC000AE92582F8E2F5F008E222E5832AF58377
:080F0C00E993F5F0A3E993223B
:100F1400BB010DC58229C582C5833AC583021178F8
:100F24005011C58229F808E5F026F618F5F0E58297
:100F340036F622BBFE11C58229F808E225F0F5F049
:100F4400F218E23582F222F8E58229F582E5832A55
:0D0F5400F58374019325F0F5F0E493382245
:100F6100F8BB0111E58229F582E5833AF583E8F0C2
:100F7100E5F0A3F0225009E92582C8F608A6F0227F
:0D0F8100BBFE09E92582C8F2E5F008F22266
:100F8E00E88FF0A4CC8BF0A42CFCE98EF0A42CFC02
:100F9E008AF0EDA42CFCEA8EF0A4CDA8F08BF0A480
:100FAE002DCC3825F0FDE98FF0A42CCD35F0FCEBDF
:100FBE008EF0A4FEA9F0EB8FF0A4CFC5F02ECD39A4
:0F0FCE00FEE43CFCEAA42DCE35F0FDE43CFC2211
:100FDD0075F008758200EF2FFFEE33FECD33CDCCCB
:100FED0033CCC58233C5829BED9AEC99E58298404E
:100FFD000CF582EE9BFEED9AFDEC99FC0FD5F0D62B
:10100D00E4CEFBE4CDFAE4CCF9A88222B800C1B954
:10101D000059BA002DEC8BF084CFCECDFCE5F0CB92
:10102D00F97818EF2FFFEE33FEED33FDEC33FCEBCB
:10103D0033FB10D703994004EB99FB0FD8E5E4F986
:10104D00FA227818EF2FFFEE33FEED33FDEC33FC73
:10105D00C933C910D7059BE99A4007EC9BFCE99A67
:10106D00F90FD8E0E4C9FAE4CCFB2275F010EF2FAC
:10107D00FFEE33FEED33FDCC33CCC833C810D707AC
:10108D009BEC9AE899400AED9BFDEC9AFCE899F8E7
:0E109D000FD5F0DAE4CDFBE4CCFAE4C8F9227A
:103B5B00C2D5E830E70FB2D5E4C39BFBE49AFAE495
:103B6B0099F9E498F8EC30E717B2D5123B911210A3
:103B7B0019E4C39BFBE49AFAE499F9E498F88003FF
:103B8B0012101930D50DE4C39FFFE49EFEE49DFD9A
:043B9B00E49CFC2288
:1010AB00EB9FF5F0EA9E42F0E99D42F0EC6480C8BC
:0610BB0064809845F0225C
:1010C100E8600FECC313FCED13FDEE13FEEF13FF0D
:0310D100D8F12231
:1010D4007401FF3395E0FEFDFCA3A3A3E0CF2FF042
:1010E400E582158270021583E0CE3EF0E58215821A
:1010F40070021583E0CD3DF0E58215827002158300
:05110400E0CC3CF022EC
:0C110900ECF0A3EDF0A3EEF0A3EFF02259
:10111500A8828583F0D083D08212112C12112C1253
:10112500112C12112CE473E493A3C583C5F0C58378
:10113500C8C582C8F0A3C583C5F0C583C8C582C824
:011145002287
:0C114600A42582F582E5F03583F58322B4
:10115200D083D082F8E4937012740193700DA3A32C
:1011620093F8740193F5828883E473740293686040
:06117200EFA3A3A380DF40
:10117800C5F0F8A3E028F0C5F0F8E5821582700202
:061188001583E038F0229F
:00000001FF
